:100000003FC0D1C258C057C056C055C054C053C0DD
:1000100052C051C050C04FC04EC04DC04CC04BC06C
:100020004AC049C048C0040309041A037700770096
:1000300077002E006F0062006400650076002E00DD
:100040006100740018034C00430044005F0044004A
:100050006900730070006C006100790012011001EA
:10006000FF000008C016DC050001010200010902C2
:10007000120001010080FA090400000000000000E5
:1000800011241FBECFE5D4E0DEBFCDBF12E0A0E655
:10009000B0E0E4E0F8E002C005900D92A235B107AF
:1000A000D9F712E0A2E5B2E001C01D92A338B10772
:1000B000E1F726D1A5C3A4CF80E58DB9089591E0DD
:1000C00098BBC298AC988FB9779BFECF84E088BB71
:1000D000C098089591E098BBC29890E195BB8FB904
:1000E000779BFECF80915702909158020196909392
:1000F000580280935702843591059CF01092580263
:100100001092570280915502909156020196909359
:10011000560280935502069724F0109256021092D0
:10012000550284E088BBC09808950F931F93182F41
:10013000062F8068C4DF802F8064C1DF10935702D0
:100140001092580200935502109256021F910F917F
:1001500008950F931F93CF93DF9380E060E0E5DF76
:1001600000E010E00BC080E0B5DF2196C435D1057A
:10017000D1F70F5F1F4F0630110519F0C0E0D0E036
:10018000F2CF80E060E0D1DFDF91CF911F910F913E
:10019000089588EE93E02CE231E0F9013197F1F710
:1001A0000197D9F7C29880E485BB88EE93E02CE2F2
:1001B00031E0F9013197F1F70197D9F780E485BB78
:1001C00084E088BB81E27BDF80EE79DF84E077DF4B
:1001D00083E175DF80E273DF8CE071DFBADF0895C1
:1001E0000F931F93CF93DF93182F8A3069F4609198
:1001F0005502709156026F5F7F4F70935602609365
:10020000550280E092DF43C044E550E08091570200
:1002100090915802481B590B4530510524F585E053
:10022000189FC0011124FC01E054F04020E030E0B0
:10023000BC016B5370408081803811F02F5F3F4FBD
:100240003196E617F707B9F74217530764F4609140
:100250005502709156026F5F7F4F70935602609304
:10026000550280E062DF85E0189FC0011124EC0197
:10027000C054D0408C010B5310408881803809F065
:1002800029DF2196C017D107C1F780E023DFDF9176
:10029000CF911F910F910895CF93DF93EC0182E5E9
:1002A00092E090936802809367028981882341F4E9
:1002B0008A81809352028B818093530282E01DC019
:1002C000813011F48A8106DF8981823011F48A81BC
:1002D000F6DE8981833009F43CDF8981843009F4BA
:1002E00058DF8981853019F48A816B811EDF89810D
:1002F000863011F48A8174DF80E0DF91CF91089518
:10030000CF93DF938FEF87BB91E098BB84BB80E5F1
:100310008DB93FDF80E062E008DF87E561DF8BE4D5
:100320005FDF84E55DDF85E45BDF82E559DF80E048
:1003300063E0FBDECBE3D2E002C0899151DF82E0D3
:10034000CE34D807D1F785E081BB88EF82BB84EF3C
:1003500091E02CE231E0F9013197F1F70197D9F7FB
:1003600011BA07D0789480E060E0DFDEA89508D06D
:10037000FDCF85B7826085BF8BB780648BBF089542
:100380001F93CF93DF9390916902935097FD87C09D
:1003900020916602809165028D3209F07EC098300E
:1003A00009F07BC0CCE0D0E0C21BD109C359DD4FBE
:1003B00083EC809359028AE580934F021092540295
:1003C0008881807621F0CE0167DF282F5DC09A8179
:1003D000109262028981882321F41092630222E044
:1003E0004DC0853019F490936A0247C08630B1F54C
:1003F0008B81813019F48CE590E004C0823041F4A7
:100400008EE690E0909368028093670222E122C01A
:100410008330F9F48A81882341F486E290E0909356
:1004200068028093670224E015C0813041F48AE2BB
:1004300090E090936802809367022AE10BC08230BB
:1004400041F484E490E0909368028093670228E18D
:1004500001C020E080E48093540216C0883021F46B
:1004600021E08CE692E00CC0893019F490936C0284
:1004700004C08A3011F421E001C020E082E692E05D
:1004800090936802809367028F81882321F48E8184
:10049000821708F4282F209350021092690280914D
:1004A0004F0284FF49C0809150028F3F09F444C03D
:1004B000182F893008F018E0811B8093500280913A
:1004C000590298E8892780935902112341F120911C
:1004D0006702309168028091540286FF0DC0AAE540
:1004E000B2E080E090E0F901E80FF91FE491ED93AC
:1004F00001961817C1F708C0912FD901EAE5F2E07B
:100500008D9181939150E1F71150812F90E01F5F01
:100510000196820F931F90936802809367028AE589
:1005200092E0612F3CD0612F6C5F6C3019F08FEF3F
:100530008093500260934F0294E180B3857031F450
:100540009150D9F710926A0210926402DF91CF9114
:100550001F910895A82FB92F8FEF9FEF1BC02D91EA
:100560008227282F22952827722F26952695272720
:10057000239526952170782F892F82272195207C1D
:10058000922F22277695279597278227769527956C
:1005900097278227615018F7809590950895DADFA4
:1005A0008D939D930895CF93CFB7CF93C395809BA1
:1005B000E9F7809B09C0809B07C0809B05C0809B9A
:1005C00003C0809B01C0A1C0DF93C0916602DD27FC
:1005D000C359DD4F809B02C0DF91EBCF2F930F9368
:1005E0001F9300B32FEF00FB20F94F933F9310B3FD
:1005F0004FEF012700FB21F93BE031C04E7F012F77
:1006000010B3216028C0102F4D7F2260000000B37E
:1006100029C04B7F2460012F000010B32BC010B302
:10062000477F28602AC04F7E00B320612CC04F7DD9
:1006300010B320622FC04F7B00B3206432C042272A
:1006400000B349934FEF0000102710FB20F910B3BF
:100650001570C9F1297F91F2012700FB21F900B340
:10066000237F89F2315058F1102710FB22F910B383
:10067000277E79F2012700FB23F92F7C81F200B35A
:10068000102710FB24F92F7971F200C010B3012755
:1006900000FB25F92F7359F200C000B3102710FB9F
:1006A00026F9223040F200C010B3012700FB27F9E1
:1006B000243028F64F77206810B30000F9CF10E4FB
:1006C0001ABF002717C03B503195C31BD04010E420
:1006D0001ABF0881033CE9F00B34D9F02091640281
:1006E0001981110F1213EDCF093641F10D3211F0BE
:1006F000013E39F700936B023F914F911F910F918B
:100700002F91DF91CAB7C6FD51CFCF91CFBFCF9107
:10071000189520916B02222379F31091690211231D
:1007200011F5343012F13093690220936502109173
:1007300066023BE0311B3093660217C000916902EC
:1007400001308CF40AE530914F0234FD10C0009363
:100750004F02C9E5D2E00FC02795A8F45150A9F483
:10076000220F0000F9CF4AE503C042ED01C0432F3C
:10077000C4E1D0E032E011B31560909A11BB02B32E
:1007800020E415E05F93012756E002BB279520F493
:10079000515021F4220FF9CF012756E000003B5AB7
:1007A00002BBD0F2279528F4515029F4220F000003
:1007B000F9CF012756E0279502BB20F4515021F4D0
:1007C000220FF9CF012756E02991332302BB21F6EE
:1007D0000A7F10916A02110FC651D04002BB11F07E
:1007E0001093640210E41ABF016011B31A7F402F06
:1007F0004A7F5F9100C000C002BB11BB42BB7CCFEF
:04080000F894FFCF9A
:1008040000000080805C808080800C000C80802848
:100814007C287C285058EC28800460100C40285414
:100824005420500C808080803844808080443880FC
:10083400808014081480801038108080C04080802C
:100844008010101080804080808080402010080438
:100854003844443880047C80808064545448804404
:100864005454288030287C20805C5454248038548C
:100874005420800464140C80285454288008545450
:100884003880288080808068808080801028448020
:1008940080282828808044281080800454140880EC
:1008A400384474543878242478807C54542880380C
:1008B400444480807C444438807C545444807C1478
:1008C40014048038445474807C10107C80447C442C
:1008D40080802040443C807C102844807C404080C0
:1008E400807C0810087C7C08107C80384444388064
:1008F4007C24241880384444B8807C2424588048BC
:1009040054542480047C0480803C40403C803C401F
:10091400300C803C4038403C6C10106C800C5050C3
:100924003C8064544C80807C448080800408102087
:1009340040447C808080080408808040404040809F
:10094400040880808030484878807C484830803073
:10095400484880803048487C80306858108010783F
:1009640014808018A4A47C807C0808708074808023
:10097400808040348080807C203044807C808080F3
:10098400807808780870780808708030484830808B
:10099400F848483080304848F88078100880805003
:1009A40058682880083C4880803840407880384027
:1009B4002018801860186018483048808018A0A05B
:1009C40078804868584880106C4480807E8080809D
:1009D40080446C1080800804080480444953504CBF
:1009E400415920494E495449414C495A4544005AB9
:0209F400FF0002
:00000001FF
